:02000000400AB4
:10008000800C02000F0C06008604A6056B0004001D
:100090000000000000000000000000000000EB0273
:1000A000480A06020F0E2900A9030F0FE901A90350
:1000B000A604060C27000B052B0309022A00780969
:1000C000080C28002A037809E802620A640C2C0054
:1000D000FA0C2B000000EB026A0A0400EC02680A2A
:1000E000E7025B0AA6050400000000000000730A96
:1000F00004008605060C2B00EB027C0A8604FE0C2D
:100100002B00000000000000EB02830A03068605B6
:10011000060C2B00EB028A0A8604FE0C2B00000062
:0A01200000000000EB02910A000845
:080800000F000A000D000E00BC
:021FFE00EE0FE4
:00000001FF
